:100000008A110A120528000009000730990083169A
:100010000510851005118312BC30A0000230A1002C
:100020008B212F20AC012C08143C031C2B28AD0184
:100030002D083B3C031C2528BC30A0000230A10049
:100040008B210130AD07031C18281F3083050130B8
:10005000AC07031C13281F3083050C282E28051419
:100060005830A0000230A1008B216E2033215D208A
:100070003321E12033218620332133217E20332197
:1000800092203321F3203321F9203321BA20332168
:10009000AB2033213321AB203321952033218A201B
:1000A00033216E2033216A20332195209030A00027
:1000B0000130A1008B21051008005721682108009C
:1000C00068215721572157210800682157216821AD
:1000D000572108006821572157210800572108009F
:1000E000572157216821572108006821682157218D
:1000F0000800572157215721572108005721572120
:1001000008005721682168216821080068215721CB
:1001100068210800572168215721572108006821CC
:10012000682108006821572108006821682168219A
:10013000080057216821682157210800682168219B
:1001400057216821080057216821572108005721AD
:10015000572157210800682108005721572168219D
:10016000080057215721572168210800572168218D
:10017000682108006821572157216821080068215B
:1001800057216821682108006821682157215721DB
:10019000080068216821682168216821080057212A
:1001A00068216821682168210800572157216821AA
:1001B00068216821080057215721572168216821AB
:1001C000080057215721572157216821080057213E
:1001D00057215721572157210800682157215721BE
:1001E000572157210800682168215721572157219D
:1001F00008006821682168215721572108006821DB
:10020000682168216821572108005721682157215A
:10021000682157216821080068216821572157214A
:10022000682168210800572157216821682157213A
:1002300057210800682157215721682157210800BC
:10024000682157215721572168210800682157212B
:100250005721572157216821080005114630A00079
:10026000A1018B21080005114630A000A1018B21BE
:100270004630A000A1018B214630A000A1018B21B6
:10028000080005114630A000A1018B214630A000D6
:10029000A1018B214630A000A1018B214630A00096
:1002A000A1018B214630A000A1018B21080005157A
:1002B000053084000230AA009930A0000230A1006D
:1002C0002D30A2000030A300C62105112D21080009
:1002D0000515053084000230AA009930A0000230D4
:1002E000A100B430A2000030A300C62105112D21C9
:1002F00008000515053084000230AA009930A000DE
:100300000230A100EE30A2000230A300C621051188
:100310002D2108008A29A008031996299D21A003F0
:10032000000000000000000000008B29A108031954
:1003300008009D21A103A0038B290C30A500A50B6B
:100340009F29000000001230A200A20BAC29AE21B0
:10035000AE21000000000800AE21A5290D30A40048
:10036000A40BB029000008001030A8020001031CF3
:10037000013EA902031C0800BD290A30A8020001A1
:10038000031C013EA902031C0800BD292A088004A1
:100390002008A8002108A900B4210130A202031CF2
:1003A000A3032A0980052008A8002108A900B42178
:0E03B000A208031DC629A308031DC6290800C4
:02400E00C431BB
:00000001FF
